:10000000830100308A001E28FC0003088301D10010
:1000100083120313A10A0319A20A07302202D13066
:1000200003192102031C1628A001A00A0B1183301A
:10003000810051088300FC0E7C0E090020308400F2
:100040004F30272083019F2C04068001840A040678
:10005000031900342428CF00D01B3728501B3F2819
:1000600050088A004F08CF0A0319D00A8200831370
:10007000501883174F08CF0A840000080800253461
:10008000643420346D34733400344234693452346F
:1000900041345A3420345034523441345434693465
:1000A0004B342034593441345034003442345534C4
:1000B00054344F344E344134203443344F344B3471
:1000C0002034453452344B3445344E3400345534A6
:1000D0005934553459344F345234533455344E34E2
:1000E0002034473441344C34693442344134003490
:1000F00020344234413453344C3441345434273462
:100100004134203442344134533449344E34203461
:100110000034203444345534523444345534523449
:1001200027344134203442344134533449344E343A
:100130002034003420345234453446344C34453471
:100140004B34533420344F344C34433445345234DC
:100150002034203400342034203443344F344B34A2
:1001600020345934413456344134533453344934AF
:100170004E34203420340034203444344134483464
:1001800041342034483449345A344C3449342034CE
:100190004F344C342034203400342034203459344B
:1001A00045344E346934443445344E342034443478
:1001B00045344E344534203420340034203459340E
:1001C0004534533469344C342034593441344E343A
:1001D00049344E3443344134203420340034203404
:1001E00020342034543445344234523469344B344E
:1001F0004C344534523420342134203420340034FB
:10020000203420342034423441345334543449347B
:100210004E3420342134213421342034203420340D
:10022000003420342034203420344D3455344B34C1
:1002300045344D344D3445344C342034203420344E
:040240002034003432
:10074E008312080083120313C1000511803E032C8F
:10075E00831203130511013003240230CC2B8312B4
:10076E004108A4004208A500A601A701A301A30AFF
:10077E000800F0000030711870070310F00D031020
:10078E00F10CF10803190800C22B83120313C200E7
:10079E000430C3005330C400C40BD32BC30BD12B76
:1007AE00C20BCF2B0800831203130515E62B42084C
:1007BE00D0004108C10A0319C20A2B2003244208A3
:1007CE00D00041082B20003803190800DE2BF4015D
:1007DE00F5010310F30CF20C031CFC2B7008F4074C
:1007EE0071080318710AF5070310F00DF10D720868
:0207FE00730482
:1008000003190034F02B83120313C300430E0F3976
:10081000F0000608F039700486008515851143083C
:100820000F39F0000608F03970048600851585112F
:100830000D30C400C40B1A2C080083120313A80047
:100840000515280E0F39F0000608F03970048600EF
:100850008515851128080F39F0000608F039700455
:100860008600851585110D30A900A90B352C0800CF
:100870008312031305110F30CC2303308600851536
:1008800085110530CC23851585112130C100C10BA0
:10089000472C851585110530CC230230860085153F
:1008A00085110D30C100C10B532C283003240830B2
:1008B00003240F3003240630032C8312A308031DE6
:1008C000652CC101C10AC201B6236D30F4004E305F
:1008D000F500C630F6004130F7002408F000250886
:1008E000F1002608F2002708F300C3273930F4008E
:1008F0003030F500F601F70174087007F800710850
:10090000F90075080318750FF9077208FA007608E0
:100910000318760FFA077308FB0077080318770FA0
:10092000FB077808A4007908A5007A08A6007B08D0
:10093000A700F1002608F0007F30F10508004730DD
:1009400083120313AE004530AF004330B00069306E
:10095000B1004B30B2004D30B3004530B4003D30F3
:10096000B5002030B600B700B800B900BA00BB002F
:10097000BC00BD00BE0183168501303086008312A5
:100980008501860107309F008316811281110110B5
:10099000811401118B178B120B11FA30CC233824E0
:1009A000AF230C3003240030A9239A30C10000305B
:1009B000C200DA234030A9237830C1000030C200E1
:1009C000DA23A001A101A201A901061EE52CAF2393
:1009D000061786130030A923DE30C1000030C200A4
:1009E000DA234030A9238930C1000030C200DA2365
:1009F0005D247008A8000330F200F3012808F0001D
:100A0000F101EE237408AC007508AD0000302D0232
:100A10004C3003192C020318112D4B30AC0703186E
:100A2000AD0AAA01AB01172DAA0A0319AB0A2D08BA
:100A30002B02031D1D2D2C082A020318252D0A3018
:100A4000CC23861E142DA901A90A290B372D0030AD
:100A5000A9235630C1000030C200DA234030A92358
:100A60000030C1000130C200DA230613E12C8617E2
:100A70000613833081008B16861E3C2D8B12AF230C
:100A80000030A923A008031DC22D003022026530CA
:100A9000031921020318512DEF30C1000030C200AC
:100AA000DA23003022026530031921020030031CD2
:100AB000652D2202C930031921020318642D11305B
:100AC000C1000130C200DA2300302202C93003190C
:100AD00021020130031C782D22022D30031921023E
:100AE0000318772DBC30C1000030C200DA2301307A
:100AF00022022D30031921020230031C8B2D220209
:100B000059300319210203188A2D4530C1000030E5
:100B1000C200DA23023022025930031921020330C5
:100B2000031C9E2D2202E9300319210203189D2D7A
:100B3000AB30C1000030C200DA2303302202E930BA
:100B400003192102031CB02D07302202D0300319F3
:100B500021020318B02D6730C1000030C200DA2333
:100B60003F30C2000030C3002108BF002208C0008F
:100B70003F30C1003630C6254030A9232E30C10099
:100B80008030DF2CCD30C1000030DF2C8312CA0052
:100B9000C80103134108C500772F4908253A031DF2
:100BA0006A2FFF30C600C701C401342FCA080319D9
:100BB000DD2D4A08840083138001480808000230B4
:100BC000C5074502840083130008682FC40AEC2D72
:100BD0000830C607FE30C6070230C507450284004C
:100BE00083130008CB00840A0008CC004418CC1FF3
:100BF000002ECB09CC09CB0A0319CC0AC703012E5E
:100C0000C4010B30C6074608F200F3014C08F1009E
:100C10004B08F0008C277008C9004608F200F30169
:100C20004B08F0004C08F1008C277408CB007508C5
:100C3000CC00CD01CD0ACE014E084C02031D222E60
:100C40004D084B02031C3F2E4608F200F3014D08ED
:100C5000F0004E08F100EE237408CD007508CE00B8
:100C6000C7031C2EC80ACA0803193D2E4A0884006F
:100C7000831320308000CA0A3F2E2030A723C703E9
:100C80004708803A7F3E0318322E441C542EC80A6F
:100C9000CA080319522E4A08840083132D3080009D
:100CA000CA0A542E2D30A7234608F200F3014D083E
:100CB000F0004E08F1008C277408CD007508CE00B6
:100CC0004D040319892E4E08F3004D08F2004C081C
:100CD000F1004B08F0008C277408F0007508F10053
:100CE0004608F200F3018C277008C700803A763E70
:100CF000031C7C2E0730C707C80ACA080319862EB2
:100D00004A08840083134708303E4F2E4708303E80
:100D1000532E0A304902031C8F2E0730C907C80A18
:100D2000CA080319992E4A08840083134908303EE3
:100D3000722F4908303E762FC80ACA080319A72E19
:100D40004A088400831320308000CA0AA92E20306C
:100D5000A723C7034708803A7E3E03189C2E023023
:100D6000C5074502840083130008C9006A2F0230BA
:100D7000C5074502840083130008CD00840A0008DB
:100D8000CE00C90149084D07CF004E08D0004F08DA
:100D90000318D00A2B2000380319D02EC90AC22EFE
:100DA000460849020318D62E4908C6004608C71B44
:100DB000022FFF3A4707031C022FC80ACA0803196B
:100DC000E82E4A088400831320308000CA0AEA2EE5
:100DD0002030A723C703D62E4E080313D0004D089A
:100DE0002B20C900CD0A0319CE0AC80ACA08031964
:100DF000002F4A088400831349088000CA0A022F82
:100E00004908A723C603460FEC2E772F4308D000CE
:100E100042082B202A3A031D142F0230C507450231
:100E2000840083130008302F4308D00042082B2091
:100E3000D03EC600C20A0319C30A4308D0004208C4
:100E40002B20C90030304902031C342F3A304902AC
:100E50000318342F0A30F1004608C0234907D03E5A
:100E6000C600C20A0319C30A4308D0004208C20AD6
:100E70000319C30A2B20C900003A0319D62D2A3AB8
:100E80000319DF2D043A0319062F763A0319E82DCA
:100E90003B3A0319AA2E073A0319E62D0B3A031918
:100EA000EA2D1C3A0319B72E063A0319EC2D0D3A18
:100EB0000319E82D30304902031C6A2F3A304902E9
:100EC00003186A2F0A30F1004708C0234907D03EB3
:100ED000C700342FC80ACA080319752F4A088400AE
:100EE000831349088000CA0A772F4908A7234308BB
:100EF0000313D0004208C20A0319C30A2B20C900F9
:100F0000C908031DCD2DCA0803198A2F4A08840079
:100F10008313800148080800F601F401F501720806
:100F20007304031900341F30F6040310F60AF20D9F
:100F3000F30D031C962FF30CF20C73087102031DC2
:100F4000A32F72087002031CAB2F7208F002730803
:100F5000031C730AF102F40DF50DF60BF61A9B2F24
:100F6000F61FB72FF409F40A0319F503F5097408FD
:100F7000F2007508F300761F0034F009F00A031937
:100F8000F103F109003484017008F8007108F900D8
:100F90007208FA007308FB00F201F301F001F1019D
:100FA0000310FB0CFA0CF90CF80C031CE52F740869
:100FB000F00775080318750FF10776080318760F08
:100FC000F20777080318770FF307780879047A0493
:100FD0007B040319F12F0310F40DF50DF60DF70D39
:100FE000D02F84080319003473088000840372082A
:100FF000800084037108800084037008800000343E
:02400E0061FF50
:00000001FF
